:020000040000FA
:0200000087284F
:0800080087288C00810183169A
:100010000313C030810508008C008101831603138F
:10002000C030810501308104831203130B110B1DB5
:1000300017288C0B162808008E00E13086050E0D5F
:100040001E398604080086132628861706138F009B
:100050000F080F0E1C2033200F081C203320E13026
:1000600086058613080001300C20861600008612D3
:1000700001300C20080011089300120894001010A1
:1000800010308D0027308E005D202520E8308D0057
:1000900003308E005D20252064308D008E015D20B0
:1000A00025200A308D008E015D20252001308D0035
:1000B0008E0110145D20252008008C010E0814020A
:1000C000031C7128031D68280D081302031C7128E6
:1000D0000E0894020D089302031C94038C0A10145A
:1000E0005E2830300C07101C203008001414120851
:1000F0009300083095003030931B31302520930D4C
:10010000950B7B28141C08001410110878288316FE
:100110000313013086058312031386120613861318
:10012000E130860504300C2003301C2033200130E0
:100130000C2008301C20332001300C2002301C2001
:10014000332001300C20283023200C3023200130B4
:10015000232008300C2092019101433025206E307D
:100160002520743025202D30252056302520613063
:1001700025206C30252075302520653025203A302B
:1001800025208B3023203B20C030232076200130D7
:0C01900091070318920A40300C20C1288F
:02400E00F13F80
:00000001FF
